:04000000FFEF08F016
:1000080000C016F001C015F06F0084FF17F06F00F4
:1000180088FF18F03901A3A775D093A773D015EC02
:1000280007F000C09DF03D01F9AB0FD0F99B010E20
:1000380002013025006E000E3121016E00C030F241
:1000480001C031F26F00A0F79DF03D01F9A70FD074
:10005800010E02013025006E000E3121016E00C034
:1000680030F201C031F215EC07F000C09DF03D01FF
:10007800F9A50FD0010E02013025006E000E3121C6
:10008800016E00C030F201C031F215EC07F000C07B
:100098009DF0A60E00019925E16E010E9A21E26EEF
:1000A8006F0087FFE1FF6F008BFFE2FF600077F2D0
:1000B800E6FF010E9525006E000E9621016E00C028
:1000C80095F001C096F0010E9925006E000E9A2158
:1000D800016E00C099F001C09AF09D510D0A09E027
:1000E800000E006E9A51005C02E19951040801E388
:1000F80009D039019397010E00019E6F000E9F6F82
:10010800996B9A6B390199A127D0A9A125D0800EA6
:10011800006E800E1A18005C02E1195000080AE20D
:10012800010E195C006E000E1A58016E00C019F01D
:1001380001C01AF0800E1A18006E800E005C02E1F1
:10014800010E195C07E23901010E1B6E000E1C6ED0
:100158009991949E3901A99116C000F015C001F03B
:0E01680060005FF0E1FF600063F0E2FF110055
:0E017600550E3A01BF6FAA0EBF6FBF91120067
:0E018400550E3A01BF6FAA0EBF6FBF81120069
:0C019200000E3D01F9BF010E006E1200CE
:10019E0002015751170802E2006A0ED35851000AA5
:1001AE00D8A4B1D05A5301E0DFDF60D0600067F908
:1001BE0000FAA5D0600067F901FAA1D0600067F9D6
:1001CE0002FA9DD0600067F903FA99D0600067F9D2
:1001DE0004FA95D0600067F905FA91D0600067F9CE
:1001EE0006FA8DD0600067F907FA89D0600067F9CA
:1001FE0008FA85D0600067F909FA81D0600067F9C6
:10020E000AFA7DD0600067F90BFA79D0600067F9C1
:10021E000CFA75D0600067F90DFA71D0600067F9BD
:10022E000EFA6DD0600067F90FFA69D0600067F9B9
:10023E0010FA65D0600067F911FA61D0600067F9B5
:10024E0012FA5DD0600067F913FA59D0600067F9B1
:10025E0014FA55D0600067F915FA51D0600067F9AD
:10026E0016FA4DD0600067F917FA49D002015751BE
:10027E00000A9CE05751010A9DE05751020A9EE088
:10028E005751030A9FE05751040AA0E05751050A3F
:10029E00A1E05751060AA2E05751070AA3E05751B1
:1002AE00080AA4E05751090AA5E057510A0AA6E028
:1002BE0057510B0AA7E057510C0AA8E057510D0AE7
:1002CE00A9E057510E0AAAE057510F0AABE0575159
:1002DE00100AACE05751110AADE05751120AAEE0C8
:1002EE005751130AAFE05751140AB0E05751150A8F
:1002FE00B1E05751160AB2E05751170AB3E00201A6
:10030E005A5301E038DF02015851010AD8A451D1E5
:10031E005A5301E029DFA4D060005FF9C0FA45D13D
:10032E0060005FF9C1FA41D160005FF9C2FA3DD1B8
:10033E0060005FF9C3FA39D160005FF9C4FA35D1B4
:10034E0060005FF9C5FA31D160005FF9C6FA2DD1B0
:10035E0060005FF9C7FA29D160005FF9C8FA25D1AC
:10036E0060005FF9C9FA21D160005FF9CAFA1DD1A8
:10037E0060005FF9CBFA19D160005FF9CCFA15D1A4
:10038E0060005FF9CDFA11D160005FF9CEFA0DD1A0
:10039E0060005FF9CFFA09D160005FF9D0FA05D19C
:1003AE0060005FF9D1FA01D160005FF9D2FAFDD099
:1003BE0060005FF9D3FAF9D060005FF9D4FAF5D096
:1003CE0060005FF9D5FAF1D060005FF9D6FAEDD092
:1003DE0060005FF9D7FAE9D060005FF9D8FAE5D08E
:1003EE0060005FF9D9FAE1D060005FF9DAFADDD08A
:1003FE0060005FF9DBFAD9D060005FF9DCFAD5D086
:10040E0060005FF9DDFAD1D060005FF9DEFACDD081
:10041E0060005FF9DFFAC9D060005FF9E0FAC5D07D
:10042E0060005FF9E1FAC1D060005FF9E2FABDD079
:10043E0060005FF9E3FAB9D060005FF9E4FAB5D075
:10044E0060005FF9E5FAB1D060005FF9E6FAADD071
:10045E0060005FF9E8FAA9D060005FF9E9FAA5D06B
:10046E0002015951000AD8B457D75951010AD8B4CC
:10047E0057D75951020AD8B457D75951030AD8B48D
:10048E0057D75951040AD8B457D75951050AD8B479
:10049E0057D75951060AD8B457D75951070AD8B465
:1004AE0057D75951080AD8B457D75951090AD8B451
:1004BE0057D759510A0AD8B457D759510B0AD8B43D
:1004CE0057D759510C0AD8B457D759510D0AD8B429
:1004DE0057D759510E0AD8B457D759510F0AD8B415
:1004EE0057D75951100AD8B457D75951110AD8B401
:1004FE0057D75951120AD8B457D75951130AD8B4ED
:10050E0057D75951140AD8B457D75951150AD8B4D8
:10051E0057D75951160AD8B457D75951170AD8B4C4
:10052E0057D75951180AD8B457D75951190AD8B4B0
:10053E0057D759511A0AD8B457D759511B0AD8B49C
:10054E0057D759511C0AD8B457D759511D0AD8B488
:10055E0057D759511E0AD8B457D759511F0AD8B474
:10056E0057D75951200AD8B457D75951210AD8B460
:10057E0057D75951220AD8B457D75951230AD8B44C
:10058E0057D75951240AD8B457D75951250AD8B438
:10059E0057D75951260AD8B457D75951270AD8B424
:1005AE0057D75951280AD8B457D702015A5301E0E8
:1005BE00E2DDA8D0020158B102D0C29001D0C280B3
:1005CE00F9D0020158B102D0C29201D0C282F2D04B
:1005DE00020158B102D0C29401D0C284EBD0020104
:1005EE0058B102D0C29601D0C286E4D0020158B1F1
:1005FE0002D0C29801D0C288DDD0020158B102D01B
:10060E00C29A01D0C28AD6D0020158B102D0C29C81
:10061E0001D0C28CCFD0020158B102D0C29E01D0FF
:10062E00C28EC8D0020158B102D0C39001D0C3808F
:10063E00C1D0020158B102D0C39201D0C382BAD048
:10064E00020158B102D0C39401D0C384B3D00201C9
:10065E0058B102D0C39601D0C386ACD0020158B1B6
:10066E0002D0C39801D0C388A5D0020158B102D0E0
:10067E00C39A01D0C38A9ED0020158B102D0C39C46
:10068E0001D0C38C97D0020158B102D0C39E01D0C5
:10069E00C38E90D0020158B102D0C49001D0C48054
:1006AE0089D0020158B102D0C49201D0C48282D046
:1006BE00020158B102D0C49401D0C4847BD002018F
:1006CE0058B102D0C49601D0C48674D0020158B17C
:1006DE0002D0C49801D0C4886DD0020158B102D0A6
:1006EE00C49A01D0C48A66D0020158B102D0C49C0B
:1006FE0001D0C48C5FD0020158B102D0C49E01D08B
:10070E00C48E58D002015751000AD8B453D757514E
:10071E00010AD8B456D75751020AD8B459D75751EF
:10072E00030AD8B45CD75751040AD8B45FD75751CF
:10073E00050AD8B462D75751060AD8B465D75751AF
:10074E00070AD8B468D75751080AD8B46BD757518F
:10075E00090AD8B46ED757510A0AD8B471D757516F
:10076E000B0AD8B474D757510C0AD8B477D757514F
:10077E000D0AD8B47AD757510E0AD8B47DD757512F
:10078E000F0A81E05751100A85E05751110A89E08E
:10079E005751120A8DE05751130A91E05751140A1E
:1007AE0095E05751150A99E05751160A9DE0575199
:0A07BE00170AA1E0FF0E006E120002
:0407C800E4DC12005B
:1007CC000B6A0A6A096A005004026F00D0FF09F034
:1007DC006F00CCFF08F0015005026F00D0FF0BF04A
:1007EC006F00CCFF0AF000500502F3500926F450BC
:1007FC000A22E86A0B2201500402F3500926F45035
:10080C000A22E86A0B2208C000F009C001F00AC0F5
:08081C0002F00BC003F0120012
:1008240054C257F255C258F256C259F2010E02018F
:060834005A6FB3DC120054
:10083A00C6DF005202E10000FBD7600053F9EAFD6F
:02084A0012009A
:10084C00FC0E3F015E175E81010EAE6E7C6A7D6A06
:02085C00120088
:10085E00086A096A100E0C6E013408360936045007
:10086E00085E0550D8A0053C095ED8B007D00450EC
:10087E0008260550D8B0053C0926D890003601361A
:06088E000C2EEAD7120057
:0808940044C254F2D0DF12004F
:10089C0044C232F245C233F246C234F247C235F298
:1008AC0048C236F249C237F24AC238F24BC239F268
:1008BC004CC22CF24DC22DF24EC22EF24FC22FF270
:1008CC0050C228F251C229F252C22AF253C22BF260
:0208DC00120008
:1008DE00086A080E0C6E003408360450085ED8B054
:0E08EE0002D00826D89000360C2EF5D7120046
:1008FC00946A948C948A9498948694849482949018
:10090C00926A050E966EFF0E936E976A040E956EA4
:10091C001B6A1C6A3901A991000E006E0201455137
:10092C00005C02E14451000807E244C219F045C2E0
:10093C001AF03901998102D039019991948E1200E3
:0C094C006F00A0F701F001C000F01200E5
:10095800AB50010F006E016A000E012244C204F080
:1009680045C205F02FDF060E046E00C002F001C07C
:1009780003F0045005E003320232039EFF0FFAD75A
:0E09880060000BF07CFF60000FF07DFF12009E
:10099600160E0201546F556B130E566F40DF170E7D
:1009A6000201546F010E556F250E566F38DF120087
:1009B6000B6A0A6A096A086A0E6A03340836045022
:1009C600085E0550D8A0053C095E0650D8A0063C36
:1009D6000A5E0750D8A0073C0B5EE86AD8A0010E55
:1009E6000E5E0336070E0C6E0334083609360A36D9
:1009F6000B360E36045003A012D0085E0550D8A060
:100A0600053C095E0650D8A0063C0A5E0750D8A0F1
:100A1600073C0B5EE86AD8A0010E0E5E11D00826D0
:100A26000550D8B0053C09260650D8B0063C0A2623
:100A36000750D8B0073C0B26E86AD8B0010E0E2640
:100A460003360C2ED1D70234083609360A360B3651
:100A56000E36045003A012D0085E0550D8A0053CFF
:100A6600095E0650D8A0063C0A5E0750D8A0073C8F
:100A76000B5EE86AD8A0010E0E5E11D0082605505E
:100A8600D8B0053C09260650D8B0063C0A260750C1
:100A9600D8B0073C0B26E86AD8B0010E0E260236FF
:100AA600070E0C6E0234083609360A360B360E3639
:100AB600045002A012D0085E0550D8A0053C095E7D
:100AC6000650D8A0063C0A5E0750D8A0073C0B5E2D
:100AD600E86AD8A0010E0E5E11D008260550D8B0DF
:100AE600053C09260650D8B0063C0A260750D8B061
:100AF600073C0B26E86AD8B0010E0E2602360C2EED
:100B0600D1D70134083609360A360B360E3604506C
:100B160002A012D0085E0550D8A0053C095E06501A
:100B2600D8A0063C0A5E0750D8A0073C0B5EE86AD0
:100B3600D8A0010E0E5E11D008260550D8B0053C8F
:100B460009260650D8B0063C0A260750D8B0073CFE
:100B56000B26E86AD8B0010E0E260136070E0C6E7B
:100B66000134083609360A360B360E36045001A013
:100B760012D0085E0550D8A0053C095E0650D8A0E4
:100B8600063C0A5E0750D8A0073C0B5EE86AD8A070
:100B9600010E0E5E11D008260550D8B0053C092678
:100BA6000650D8B0063C0A260750D8B0073C0B269C
:100BB600E86AD8B0010E0E2601360C2ED1D70034C5
:100BC600083609360A360B360E36045001A012D006
:100BD600085E0550D8A0053C095E0650D8A0063C24
:100BE6000A5E0750D8A0073C0B5EE86AD8A0010E43
:100BF6000E5E11D008260550D8B0053C09260650D1
:100C0600D8B0063C0A260750D8B0073C0B26E86A3F
:100C1600D8B0010E0E260036070E0C6E00340836CC
:100C260009360A360B360E36045000A012D0085E7E
:100C36000550D8A0053C095E0650D8A0063C0A5EC1
:100C46000750D8A0073C0B5EE86AD8A0010E0E5EDE
:100C560011D008260550D8B0053C09260650D8B054
:100C6600063C0A260750D8B0073C0B26E86AD8B0DF
:100C7600010E0E2600360C2ED1D700B00ED0045031
:100C860008260550D8B0053C09260650D8B0063CC3
:0C0C96000A260750D8B0073C0B261200BD
:100CA200020144510308D8A0446B45510308D8A05F
:100CB200456BF00E3D01F217020144513D01F21362
:100CC200300EF21345C200F000360090003600905C
:100CD20000360090003600900050F413F38F12009B
:100CE2006000EBF8F6FF6000EFF8F7FF6000F3F842
:100CF200F8FF09006F00D4FF01F00150000815E26F
:100D02006000EBF8F6FF6000EFF8F7FF6000F3F821
:100D1200F8FF09006F00D4FF44F2BBDD010E0201AF
:0C0D22003A27000E3B233C23DBD71200D5
:100D2E0033DE2A0E0201446F0E0E456F000E466F23
:100D3E00000E476F940E486F080E496F440E4A6FAF
:100D4E00020E4B6FFF0E4C6FFF0E4D6F000E4E6F6F
:100D5E00000E4F6FC80E506F070E516F000E526F80
:0E0D6E00000E536F94DD446B456B94DF120052
:100D7C003901C06BC16BC26BCA6A020E3A01406F7B
:100D8C00A70EC26EC284C296439DBA96FC0E416FEA
:100D9C00506BCB6AFF0EC36EFF0E516F3E01BC6BE6
:100DAC00B86BC382C3843901C06BCC6A3A01606BE7
:100DBC00800EC46EC49ABC9AC296BA963E01C16BA0
:0C0DCC00C18FC183C1913A01636B12001A
:100DD800220E0C6E086A096A0A6A0B6A0C06D8B4F5
:100DE8001FD0D8900B320A3209320832033202324D
:100DF80001320032D8A0F2D70C06D8B409D004507A
:100E080008260550092206500A2207500B22EAD765
:100E1800045008260550092206500A2207500B22C2
:020E28001200B6
:040E2A0090DD120045
:100E2E00390199917C6A0201446B456B60DD7E8EBF
:100E3E003901A9B167D0A4B501D0FDD7A4950001A1
:100E4E0090512026915121229251222293512322F8
:100E5E003F0E2214006EAB0E0024F66E1F0EF76EC0
:100E6E00000EF722000EF86E000EF8226F00DBFF68
:100E7E00F6FF6F00DFFFF7FF6F00E3FFF8FF0900DB
:100E8E006F00D4FF3AF28F51040A02E102013A6B6D
:100E9E0000018B5124268C5125228D5126228E51F4
:100EAE0027223F0E2614006E6B0E0024F66E1F0EC8
:100EBE00F76E000EF722000EF86E000EF8226F008D
:100ECE00DBFFF6FF6F00DFFFF7FF6F00E3FFF8FFBA
:100EDE0009006F00D4FF00F0005002013A25026EA7
:100EEE0002C03AF202C000F00032009E00C03AF298
:100EFE000E0E002600C03AF200C044F2000E456FFE
:080F0E0024DD96D77E9E12003F
:100F160002013E6B050E3E5D0AE23E513C25E16E46
:100F2600000E3D21E26E200EE66E3E2BF3D73E51BB
:100F36003C25E16E000E3D21E26EE66A3E073E511B
:100F46003C253F6F000E3D21406F0A0E046E000ED9
:100F5600056E3AC200F03BC201F07EDC08C000F02C
:100F660009C001F0300E00266000FFF8E1FF6000C6
:100F760003F9E2FF600003F0E6FF0A0E046E000EBE
:100F8600056E3AC200F03BC201F066DC00C03AF2E0
:100F960001C03BF2000E011802E1000E001801E14B
:080FA60002D03E07CCD7120077
:100FAE0009006F00D7FFE6FF0006FAE10106F8E13F
:020FBE0012001F
:100FC000016A026A800E0218006E800E000A005C40
:100FD00002E1810E015C10E2A60E0124E16E010E19
:100FE0000220E26E6F0087FFE1FF6F008BFFE2FFE0
:100FF000E66A014A022AE6D70101A66B0001996B55
:101000009A6B976B986B956B966B9E6B9F6B3D0184
:10101000F289F96BFA6B00019E6B9F6B9D6B390136
:061020009387D28E12003E
:101026000201406B416B000E415D02E10A0E405D1C
:101036000BE240513E25E16E41513F21E26E200E0A
:10104600E66E404B412BEFD740513E25E16E4151B4
:101056003F21E26EE66A010E405F000E415B4051A1
:101066003E25426F41513F21436F0A0E046E000E2A
:10107600056E066E076E3AC200F03BC201F03CC236
:1010860002F03DC203F094DC08C000F009C001F094
:101096000AC002F00BC003F0300E002660000BF908
:1010A600E1FF60000FF9E2FF600003F0E6FF0A0EC1
:1010B600046E000E056E066E076E3AC200F03BC265
:1010C60001F03CC202F03DC203F072DC00C03AF20D
:1010D60001C03BF202C03CF203C03DF2000E046EBA
:1010E600031808E10450021805E10450011802E152
:1010F6000050000A01E105D0010E405F000E415B81
:04110600AED712004E
:10110A007E6A7E987E867E847E927E903F015E9382
:08111A005E817F6A7E8E1200E7
:101122000D0E0201446F4AEC04F00A0E0201446FF4
:061132004AEC04F012007B
:10113800120E0201546F556B090E566F12EC04F033
:0611480026EC04F0120089
:10114E006000EBF8E9FF6000EFF8EAFFEE500008F0
:10115E000FE26000EBF8E9FF6000EFF8EAFF6F00C6
:10116E00B8FF44F24AEC04F002013A4B3B2BE8D7AD
:02117E0012005D
:1011800002013D6B030E3D5D0AE23D513B25E16EE0
:10119000000E3C21E26E200EE66E3D2BF3D73D5152
:1011A0003B25E16E000E3C21E26EE66A3D073D51B3
:1011B0003B253E6F000E3C213F6F0A0E046E3AC283
:1011C00000F06FEC04F008C000F0300E0026600064
:1011D000FBF8E1FF6000FFF8E2FF600003F0E6FFCC
:1011E0000A0E046E3AC200F06FEC04F000C03AF24E
:0E11F0000050000A01E102D03D07D9D71200DD
:1011FE005AEC12F0600E3901D96FDB6BDD6B080E05
:10120E00DF6FDE6B6E0070F71DF0B1DD1E6A1F6AB8
:10121E00196A1A6A0101216B226B000E225D02E12E
:10122E00080E215D11E2BA78150E0B6E4B0E0C6E88
:10123E00BE0E0D6E0D2EFED70C2EFCD70B2EFAD732
:10124E000000214B222BE9D7216B226B000E225D71
:10125E0002E1800E215D10E2A10E2125E16E000E4D
:10126E002221E26E6F0087FFE1FF6F008BFFE2FF2E
:10127E00E66A214B222BEAD7BA98216B226B000E1D
:10128E00225D02E17F0E215D10E2250E2125E16E29
:10129E00010E2221E26E6F0087FFE1FF6F008BFFD0
:1012AE00E2FFE66A214B222BEAD7216B226B000E5E
:1012BE00225D02E1810E215D10E2A60E2125E16E76
:1012CE00010E2221E26E6F0087FFE1FF6F008BFFA0
:1012DE00E2FFE66A214B222BEAD7250E236F010E81
:1012EE00246FBBEC00F0156B146B130E166F170EFC
:1012FE00E56FC2EC00F08A0E3D01F56F000EF66F41
:10130E00F28F0EDD2A0E0201446F0E0E456F000E97
:10131E00466F000E476F940E486F080E496F440ECD
:10132E004A6F020E4B6FFF0E4C6FFF0E4D6F000E8D
:10133E004E6F000E4F6FC80E506F070E516F000E9E
:10134E00526F000E536F4EEC04F0520E0B6E2B0EBE
:10135E000C6E000E0D6E0D2EFED70C2EFCD70B2E26
:10136E00FAD700000C0E446F4AEC04F0190E02017D
:10137E003A6F240E3B6F000E3C6FACDC0101216B0B
:10138E00226B000E225D02E10A0E215D24E2030EA5
:10139E00006E000E016E21C104F022C105F0E6ECD4
:1013AE0003F0690E0024E96E000E0120EA6E6F0054
:1013BE00A7FFE9FF6F00ABFFEAFF6F00B8FF3AF23D
:1013CE006F00B8FF3BF26F00B8FF3CF283DC010107
:1013DE00214B222BD6D79EDE8A0E02013A6F230EA8
:1013EE003B6F000E3C6F76DC6F0E02013A6F230EE0
:1013FE003B6F000E3C6F6EDC540E02013A6F220EF4
:10140E003B6F000E3C6F66DC7F0E02013A6F220EC0
:10141E003B6F000E3C6F5EDC7DDE70DEAC98AC9AEE
:10142E00AC9CFF0EAB6E81DE7E9EAC9ED60E020194
:10143E003A6F230E3B6F000E3C6F4CDCCBB210D0DC
:10144E00D20E02013A6F220E3B6F000E3C6F42DC51
:10145E00BBEC00F0126B090E146FC2EC00F00FD053
:10146E00C20E02013A6F210E3B6F000E3C6F32DC52
:10147E00BBEC00F0146B090E126FC2EC00F07E8E06
:10148E00AC8E7E882B0E02013A6F200E3B6F000E43
:10149E003C6F20DC006A7EB8002A0050300F02013B
:1014AE00446F4AEC04F07EB809D0ED0E02013A6F9B
:1014BE00230E3B6F000E3C6F0DDC08D0030E0201B5
:1014CE003A6F240E3B6F000E3C6F04DC23DE0001EE
:1014DE009B6B9C6B580E02013A6F210E3B6F000EF8
:1014EE003C6F71EC06F0100E0001946FF00E945DDF
:1014FE002AE294C03AF2A10E02013B6F000E3C6F3D
:10150E0038DE830E3A6F240E3B6F000E3C6F71EC8B
:10151E0006F0A10E02013A6F000E3B6F11DEFADDEE
:10152E007C6A600053F27DFFBA86150E0C6EC60EF5
:10153E000D6E0D2EFED70C2EFCD70000BA96100E97
:10154E0000019427D3D7E6DDBE0E02013A6F230EBB
:10155E003B6F000E3C6F71EC06F0060E0201446FFD
:10156E00000E456F7EEC04F09981D28E000E1C1891
:10157E0002E1000E1B1813E12E0E0201446F4AEC1D
:10158E0004F0150E0B6E4B0E0C6EBE0E0D6E0D2E68
:10159E00FED70C2EFCD70B2EFAD70000E7D7BADDFC
:1015AE007E98FA0E02013A6F220E3B6F000E3C6FD0
:1015BE0071EC06F06A0E02013A6F200E3B6F000EC0
:1015CE003C6F71EC06F0E60E02013A6F200E3B6F97
:1015DE00000E3C6F71EC06F000018F6BB70E906F32
:1015EE00B60E916F000E926F936F8A6BEF0E8B6F2C
:1015FE003C0E8C6F010E8D6F000E8E6F980E0201D9
:10160E003A6F240E3B6F000E3C6F71EC06F08FC0EC
:10161E0000F0000E016E003600900136590E0024C7
:10162E00E96E000E0120EA6E6F00A7FFE9FF6F0062
:10163E00ABFFEAFF6F00B8FF3AF26F00B8FF3BF264
:10164E00A10E02013C6F000E3D6F5EDCA10E3A6FE3
:10165E00000E3B6F75DD5B0E02013A6F240E3B6F81
:10166E00000E3C6F71EC06F08AC000F0000E016EA9
:10167E00003600900136610E0024E96E000E012046
:10168E00EA6E6F00A7FFE9FF6F00ABFFEAFF6F0086
:10169E00B8FF3AF26F00B8FF3BF2A10E02013C6FA9
:1016AE00000E3D6F31DCA10E3A6F000E3B6F48DD30
:1016BE008C0E02013A6F240E3B6F000E3C6F71ECE4
:1016CE0006F0BA8617EC07F0BA96A30E0B6E570EFD
:1016DE000C6E020E0D6E0D2EFED70C2EFCD70B2EA1
:1016EE00FAD7000017DDF30E02013A6F210E3B6FA1
:1016FE00000E3C6F71EC06F000018F6B040E8F5DD7
:10170E00D8B053D18A6B040E8A5DD8B04CD18FC03D
:10171E0021F1000E0101226F21372237219121374D
:10172E002237219100018A5101012127000E222327
:10173E00200E0201446F4AEC04F0280E010121250F
:10174E00E96E000E2221EA6E6F00A7FFE9FF6F001F
:10175E00ABFFEAFF6F00B8FF44F24AEC04F0200E34
:10176E000201446F4AEC04F0050E006E000E016E8D
:10177E00026E036E21C104F022C105F0000E066E4A
:10178E00076EECEC06F0D00E002402013A6F1E0E2E
:10179E0001203B6F000E02203C6F71EC06F0090E2B
:1017AE000201446F4AEC04F0A20E02013A6F240EBD
:1017BE003B6F000E3C6F71EC06F08FC000F0000E18
:1017CE00016E003600900136590E0024E96E000EAF
:1017DE000120EA6E6F00A7FFE9FF6F00ABFFEAFF83
:1017EE006F00B8FF3AF26F00B8FF3BF2A10E020194
:1017FE003C6F000E3D6F8BEC07F0A10E3A6F000EA2
:10180E003B6F9EDC6F0E02013A6F240E3B6F000E93
:10181E003C6F71EC06F08AC000F0000E016E0036CF
:10182E0000900136610E0024E96E000E0120EA6E72
:10183E006F00A7FFE9FF6F00ABFFEAFF6F00B8FF75
:10184E003AF26F00B8FF3BF2A10E02013C6F000EA0
:10185E003D6F8BEC07F0A10E3A6F000E3B6F70DC04
:10186E00510E02013A6F240E3B6F000E3C6F71EC6D
:10187E0006F08FC000F0000E016E003600900136AB
:10188E00003600900136390E0024E96E000E01205C
:10189E00EA6E6F00A7FFE9FF6F00ABFFEAFF6F0074
:1018AE00B8FF00F06F00B8FF01F06F00B8FF02F054
:1018BE006F00B8FF03F000C090F001C091F002C0BD
:1018CE0092F003C093F000C03AF201C03BF202C0A6
:1018DE003CF203C03DF2A10E02013E6F000E3F6FBF
:1018EE0013EC08F0A10E3A6F000E3B6F29DC920E3E
:1018FE0002013A6F240E3B6F000E3C6F71EC06F046
:10190E008AC000F0000E016E0036009001360036DF
:10191E0000900136490E0024E96E000E0120EA6E99
:10192E006F00A7FFE9FF6F00ABFFEAFF6F00B8FF84
:10193E0000F06F00B8FF01F06F00B8FF02F06F000B
:10194E00B8FF03F000C08BF001C08CF002C08DF028
:10195E0003C08EF000C03AF201C03BF202C03CF26E
:10196E0003C03DF2A10E02013E6F000E3F6F13EC5D
:10197E0008F0A10E3A6F000E3B6FA7EC08F091EC49
:10198E0008F017EC07F0520E0B6E2B0E0C6E000EBD
:10199E000D6E0D2EFED70C2EFCD70B2EFAD7000097
:1019AE0000018A2BB0D68F2BA9D691EC08F08F0EA2
:1019BE0002013A6F210E3B6F000E3C6F71EC06F088
:1019CE00370E02013A6F230E3B6F000E3C6F71EC27
:1019DE0006F0EB0E02013A6F1F0E3B6F000E3C6FCE
:1019EE0071EC06F091EC08F000018F6B8A6B006AC7
:1019FE00016A390E0024E96E000E0120EA6E6F00B6
:101A0E00A7FFE9FF6F00ABFFEAFF6F00B8FF90F092
:101A1E006F00B8FF91F06F00B8FF92F06F00B8FF43
:101A2E0093F0006A016A490E0024E96E000E01204F
:101A3E00EA6E6F00A7FFE9FF6F00ABFFEAFF6F00D2
:101A4E00B8FF8BF06F00B8FF8CF06F00B8FF8DF011
:101A5E006F00B8FF8EF017EC07F0E0EC07F0520EB7
:101A6E000B6E2B0E0C6E000E0D6E0D2EFED70C2E69
:101A7E00FCD70B2EFAD70000000E00019F1902E1D1
:101A8E00010E9E19D8A48CD00101A6514F0A3DE13A
:101A9E00A7C1A0F0300E0001A05D006E00C0A5F140
:101AAE000A0E00026F00CCFF01F001C0A5F1A8C123
:101ABE00A0F0300EA05D006E0050012601C0A5F111
:101ACE00800E0118006E800E3F0A005C1EE2600060
:101ADE0097F6DEF9400E02013A6F240E3B6F000EB0
:101AEE003C6F71EC06F06E0078F73AF2A10E02012F
:101AFE003B6F000E3C6FC0EC08F0A10E3A6F000E6B
:101B0E003B6FA7EC08F091EC08F00101A651520AC8
:101B1E0047E1A851430A44E1790E02013A6F240EBF
:101B2E003B6F000E3C6F71EC06F0A7C1A0F0300EBB
:101B3E000001A05D016E01C0A5F1800E0118006EBE
:101B4E00800E040A005C2CE2A5C18FF0300E01015C
:101B5E00A5250201446F4AEC04F0A9C1A0F0300E95
:101B6E000001A05D016E01C0A5F1800E0118006E8E
:101B7E00800E040A005C12E2A5C18AF0B00E0201CA
:101B8E003A6F240E3B6F000E3C6F71EC06F0300E78
:101B9E0000018A250201446F4AEC04F091EC08F032
:101BAE008FC021F1000E0101226F213722372191C2
:101BBE0021372237219100018A5101012127000E80
:101BCE002223200E0201446F4AEC04F0280E01017C
:101BDE002125E96E000E2221EA6E6F00A7FFE9FFB4
:101BEE006F00ABFFEAFF6F00B8FF44F24AEC04F05F
:101BFE00200E0201446F4AEC04F0050E006E000E3A
:101C0E00016E026E036E21C104F022C105F0000EBA
:101C1E00066E076EECEC06F0D00E002402013A6F51
:101C2E001E0E01203B6F000E02203C6F71EC06F081
:101C3E00200E0201446F4AEC04F0090E0201446FBB
:101C4E004AEC04F0A70E02013A6F240E3B6F000E11
:101C5E003C6F71EC06F08FC000F0000E016E003686
:101C6E0000900136590E0024E96E000E0120EA6E36
:101C7E006F00A7FFE9FF6F00ABFFEAFF6F00B8FF31
:101C8E003AF26F00B8FF3BF2A10E02013C6F000E5C
:101C9E003D6F8BEC07F0A10E3A6F000E3B6FA7EC79
:101CAE0008F0650E02013A6F240E3B6F000E3C6F7A
:101CBE0071EC06F08AC000F0000E016E0036009046
:101CCE000136610E0024E96E000E0120EA6E6F00EF
:101CDE00A7FFE9FF6F00ABFFEAFF6F00B8FF3AF214
:101CEE006F00B8FF3BF2A10E02013C6F000E3D6F7C
:101CFE008BEC07F0A10E3A6F000E3B6FA7EC08F0CD
:101D0E00AC0E02013A6F240E3B6F000E3C6F71EC6D
:101D1E0006F08FC000F0000E016E00360090013606
:101D2E00003600900136390E0024E96E000E0120B7
:101D3E00EA6E6F00A7FFE9FF6F00ABFFEAFF6F00CF
:101D4E00B8FF90F06F00B8FF91F06F00B8FF92F0FF
:101D5E006F00B8FF93F08AC000F0000E016E0036DF
:101D6E0000900136003600900136490E0024E96ECF
:101D7E00000E0120EA6E6F00A7FFE9FF6F00ABFFB8
:101D8E00EAFF6F00B8FF8BF06F00B8FF8CF06F00AA
:101D9E00B8FF8DF06F00B8FF8EF091EC08F0BA86A8
:0A1DAE0017EC07F0BA9659D6FFD7DC
:1024B40010EE19F0050E006E010E016E9D0EF66E03
:1024C400240EF76E000EF86ED7EC07F010EE28F02D
:1024D400620E006E010E016EB80EF66E1D0EF76EE2
:1024E400000EF86ED7EC07F010EE1EF0020E006E30
:1024F400010E016E060EF66E000EF76E000EF86EFB
:06250400D7EC07F0120005
:020006000000F8
:101DB800313233413435364237383943302A2344B7
:011DC800001A
:101DC900B7B60000DAC9000059DF0000ADF600001F
:101DD900EF3C0100395E01003083010015AC0100C0
:081DE900B90202035403AD032B
:081DF100B9043805C5056106BF
:101DF900791E002D24002021002422001A1E00A58E
:101E09002300201F00532300AA2200A82000192321
:011E190000C8
:101E1A0020436F6E66696720626974203A205031E8
:101E2A00384632374B34325F466F73635F496E749C
:101E3A0065726E655F4C65676163795F696E74652B
:101E4A007272757074735F313678345F504C4C5FC0
:101E5A0036344D487A2E6366677363680D0A2046E6
:0F1E6A004F53433A36342E30204D487A0D0A003C
:101E7900204469726563746F7279203A433A5C5FF2
:101E89004D696B726F435C5F4D657350726F6A6524
:101E990074735F4D696B726F435C5F3138463237DB
:101EA9004B34325F526F6D616E5F426C61636B5F81
:101EB90044544D465F47656E657261746575725F1E
:071EC900323032320D0A0035
:101ED0004C4C4C48004C4C484C004C4C484800483A
:101EE000484C48004C484C4C004C484C48004C482E
:101EF000484C004848484C004C48484800484C4C26
:101F00004C00484C4C48004848484800484C484C15
:101F100000484C48480048484C4C004C4C4C4C0045
:101F200020536F75726365203A205049433138461B
:101F300032374B34325F526F6D616E5F426C61635A
:101F40006B5F44544D465F47656E6572617465759D
:101F5000725F5243325F6F755F5243345F3230328B
:0B1F6000325F313230362E630D0A0074
:101F6B0032363B4044494D5155585B5D5F6162636E
:101F7B00636362615F5D5B5855514D4944403B362D
:101F8B00322D28231F1A16120E0B0806040201000D
:101F9B00000001020406080B0E12161A1F23282D2F
:101FAB00272A2E3235393C3F424447484A4B4C4D49
:101FBB004D4D4C4B4A484744423F3C3935322E2A13
:101FCB0027231F1B1814110E0B0906050302010012
:101FDB0000000102030506090B0E1114181B1F2329
:101FEB00206D6F64696620636F646520766961207C
:101FFB00736169736965206465205278437820208A
:10200B002852616E67E96520657420436F6C6F6EB3
:10201B006E6520646520746F75636865290D0A0011
:10202B00204649475552452032332D353A205057DB
:10203B004D2031302D42495420414C49474E4D459E
:10204B004E54207061676520333439200D0A2045CA
:0F205B007461742062697420464D54203D20004A
:10206A002020202020706F757220706F75766F693E
:10207A00722072657574696C69736572206C61206F
:10208A00666F6E6374696F6E204D696B726F432061
:0E209A0028656E20382062697473290D0A00D3
:1020A8002050574D31207375722052433220706191
:1020B800722064656661757420207369205242310C
:1020C8003D31202C205541525431203A205278205D
:0E20D80052433720205458205243360D0A0040
:1020E6002064656661756C74207374617274696EC0
:1020F600672076616C75657320666F7220746865FB
:102106002044544D462064726F773D3020616E64E2
:0A2116002064636F6C3D300D0A0079
:102120002050726F6A6574203A5049433138463204
:10213000374B34325F526F6D616E5F426C61636B1F
:102140005F44544D465F47656E6572617465757294
:082150005F323032320D0A004B
:102158002054657374204343503120656E206D6FA1
:1021680064652050574D206173736F6369E920E0FF
:1021780020544D52322C2070776D20313620E020CB
:07218800323234200D0A0081
:10218F00204F534354554E4520616A7573746162F5
:10219F006C652076696120636465204F7878202014
:1021AF002061766563207878203020E02036322059
:0321BF000D0A0006
:1021C2002043686F6978205242313D31203D3E50B4
:1021D200574D2073757220736F7274696520524374
:1021E20032287061722064656661757421290D0A56
:0121F20000EC
:1021F3002047656E65726174696F6E206465732034
:10220300313620636F6465732044544D4620206942
:102213006E74657276616C6C6520317365630D0A4B
:0122230000BA
:102224002067656E65726174696F6E2064652073E2
:102234006F6E732044544D4620766961203862697C
:1022440074732050434D206F75747075740D0A00BB
:1022540020526F77203A2020203639372020202042
:1022640037373020202020383532202020203934C0
:0B22740031202020204F46460D0A00BC
:10227F0020436F6C203A202031323039202020311A
:10228F003333362020203134373720202031363376
:0B229F0033202020204F46460D0A008F
:1022AA00207573616765206465206C27416C676FD0
:1022BA00726974686D6520646520526F6D616E2065
:0822CA00426C61636B0D0A0018
:1022D2002043686F6978205242313D30203D3E20D4
:1022E20050574D202073757220736F727469652088
:0822F20020524334200D0A00C4
:1022FA002052656D69736520464D542062697420C9
:0F230A0020E0205A65726F20212121200D0A004A
:1023190043686F69782050574D3120737572205288
:0E2329004334207369205242313D300D0A00CA
:1023370020636F646520746F756368652031207052
:0C2347006172206465666175740D0A0007
:102353002031384632374B343220554152543120E4
:0C2363003139323030206264730D0A0002
:10236F002053656C65637420746865203220445473
:0B237F004D4620746F6E65730D0A0060
:10238A002053696E65776176652044544D4620670F
:0B239A00656E657261746F720D0A00C1
:1023A50020456570726F6D3A206E6F742075736588
:0923B50064202E2E2E2E0D0A00CC
:1023BE0020496E69742054696D65723620E02033B1
:0823CE0020736563203A200032
:1023D60020496E69742050574D3120617420363281
:0723E600353030487A200079
:1023ED0020416C69676E656D656E7420E0206472C6
:0623FD006F697465200009
:1024030020416C69676E656D656E7420E0206761BD
:06241300756368652000FE
:102419000D0A2050726573656E746174696F6E2060
:042429003A0D0A005E
:10242D00204D696B726F432070726F20372E3630DE
:03243D000D0A0085
:102440000D0A204E6577204F534354554E453D208D
:01245000008B
:0A24510020487A20202050413D0071
:0A245B0020487A202C2046323D0074
:0A24650020487A202C2046323D006A
:0A246F0020487A202C2046323D0060
:0A2479000D0A204E6F74652052001A
:092483002070776D31203D20002E
:06248C0020487A0D0A0051
:06249200202050423D0035
:052498002046313D006B
:02249D0000003D
:02249F0000003B
:0124A100003A
:0524A2002046313D0061
:0524A7002046313D005C
:0424AC0020487A004A
:0324B000204300C6
:020000040030CA
:0A000000242925A70B3F9F0F0100E4
:00000001FF
